:1000000000308A007D2800000230AB008316851581
:100010008312851D0D280230AB0783160516831247
:10002000051E14280430AB07831685168312851E1F
:100030001B280830AB072B08A100080083169B0182
:100040009C131C141A088312A600A5010130831604
:100050009B009C131C141A088312A5070318A60AF8
:10006000C52883168510831285142408A40AAB00C2
:100070002B0883169B009C131C141A088312A900DA
:10008000290F462804202108A40035282408A40AA2
:10009000AB002B0883169B009C131C141A088312B8
:1000A000AA002A089300831605148312051C6128F0
:1000B0000030A100063892002908831692006828B3
:1000C00083120030A10004389200290883169200A0
:1000D0008312C6282C308400000803197C280230C3
:1000E000A100A001A00B7228A10B71289730A000DD
:1000F000A00B7828800B6F28080084011F3083052F
:10010000713083168F000F0883121F1383161F1080
:100110009F101F119F110730831299001F13831620
:100120001F109F101F119F111F129F121F13831268
:100130009F131F1483160108C739083881008312E2
:1001400090010030A1009200003083169200073029
:100150008312990083160508850006308312A000DB
:10016000A00BB028000019088C118316990171307A
:100170008F000F08831204202108A40083160511A4
:10018000831205110C3095001E2831280230A90079
:100190009630AC006A20A90BC828831685108312FC
:1001A00085102C302502A9002608AA000130031C66
:1001B0000230AA022A08AB00AB0AAB030319E428F9
:1001C000FF30AC006A20DD282908AC006A20C52871
:0201D0006300CA
:104200000D00AC00630031005E002F005A002D004D
:1042100056002B00520029004F0027004C002600BA
:10422000440022003E001F0038001C0034001A0029
:10423000300018002C0016002A001500270013007B
:1042400025001200230011002100100020000100B1
:04425000FF00FF006C
:02400E00D530AB
:00000001FF
